******************************************************************************
                  TI ARM Linker PC v16.9.1                     
******************************************************************************
>> Linked Wed Mar 29 10:57:43 2017

OUTPUT FILE NAME:   <hello.out>
ENTRY POINT SYMBOL: "_c_int00"  address: 000009e9


MEMORY CONFIGURATION

         name            origin    length      used     unused   attr    fill
----------------------  --------  ---------  --------  --------  ----  --------
  FLASH                 00000000   00100000  00001104  000feefc  R  X
  SRAM                  20000000   00040000  00000220  0003fde0  RW X


SEGMENT ALLOCATION MAP

run origin  load origin   length   init length attrs members
----------  ----------- ---------- ----------- ----- -------
00000000    00000000    00001104   00001104    r-x
  00000000    00000000    00000200   00000200    r-- .intvecs
  00000200    00000200    00000be4   00000be4    r-x .text
  00000de4    00000de4    000002fc   000002fc    r-- .const
  000010e0    000010e0    00000024   00000024    r-- .cinit
20000000    20000000    00000220   00000000    rw-
  20000000    20000000    00000200   00000000    rw- .stack
  20000200    20000200    00000020   00000000    rw- .data


SECTION ALLOCATION MAP

 output                                  attributes/
section   page    origin      length       input sections
--------  ----  ----------  ----------   ----------------
.intvecs   0    00000000    00000200     
                  00000000    00000200     startup_ccs.obj (.intvecs)

.text      0    00000200    00000be4     
                  00000200    00000200     driverlib.lib : sysctl.obj (.text:SysCtlClockFreqSet)
                  00000400    000001ea     uartstdio.obj (.text:UARTvprintf)
                  000005ea    00000132     driverlib.lib : gpio.obj (.text:GPIOPadConfigSet)
                  0000071c    000000f8     spi_master.obj (.text:main)
                  00000814    0000009c     rtsv7M4_T_le_v4SPD16_eabi.lib : memcpy_t2.obj (.text)
                  000008b0    00000070                                   : autoinit.obj (.text)
                  00000920    00000068                                   : copy_decompress_lzss.obj (.text:decompress:lzss)
                  00000988    00000060     uartstdio.obj (.text:UARTStdioConfig)
                  000009e8    00000054     rtsv7M4_T_le_v4SPD16_eabi.lib : boot.obj (.text)
                  00000a3c    00000054                                   : exit.obj (.text)
                  00000a90    0000004c     spi_master.obj (.text:InitConsole)
                  00000adc    0000004c     rtsv7M4_T_le_v4SPD16_eabi.lib : cpy_tbl.obj (.text)
                  00000b28    00000048     driverlib.lib : gpio.obj (.text:GPIOPinConfigure)
                  00000b70    00000048     uartstdio.obj (.text:UARTwrite)
                  00000bb8    00000048     driverlib.lib : sysctl.obj (.text:_SysCtlFrequencyGet)
                  00000c00    00000040     rtsv7M4_T_le_v4SPD16_eabi.lib : u_divt2.obj (.text)
                  00000c40    0000003c     driverlib.lib : ssi.obj (.text:SSIConfigSetExpClk)
                  00000c7c    00000034                   : sysctl.obj (.text:SysCtlPeripheralEnable)
                  00000cb0    0000002a                   : gpio.obj (.text:GPIODirModeSet)
                  00000cda    00000002     startup_ccs.obj (.text:FaultISR)
                  00000cdc    00000020     driverlib.lib : sysctl.obj (.text:_SysCtlMemTimingGet)
                  00000cfc    0000001a     uartstdio.obj (.text:UARTprintf)
                  00000d16    00000002     startup_ccs.obj (.text:IntDefaultHandler)
                  00000d18    00000018     rtsv7M4_T_le_v4SPD16_eabi.lib : args_main.obj (.text)
                  00000d30    00000014                                   : _lock.obj (.text)
                  00000d44    00000012     driverlib.lib : gpio.obj (.text:GPIOPinTypeSSI)
                  00000d56    00000012                   : gpio.obj (.text:GPIOPinTypeUART)
                  00000d68    00000012                   : ssi.obj (.text:SSIAdvDataPutFrameEnd)
                  00000d7a    00000012                   : ssi.obj (.text:SSIDataGetNonBlocking)
                  00000d8c    0000000e     rtsv7M4_T_le_v4SPD16_eabi.lib : copy_decompress_none.obj (.text:decompress:none)
                  00000d9a    0000000c     driverlib.lib : ssi.obj (.text:SSIAdvModeSet)
                  00000da6    0000000a                   : ssi.obj (.text:SSIAdvFrameHoldEnable)
                  00000db0    0000000a                   : ssi.obj (.text:SSIDataPut)
                  00000dba    0000000a                   : ssi.obj (.text:SSIEnable)
                  00000dc4    00000008                   : ssi.obj (.text:SSIBusy)
                  00000dcc    00000006     startup_ccs.obj (.text:ResetISR)
                  00000dd2    00000006     driverlib.lib : uart.obj (.text:UARTClockSourceSet)
                  00000dd8    00000004     rtsv7M4_T_le_v4SPD16_eabi.lib : pre_init.obj (.text)
                  00000ddc    00000002     startup_ccs.obj (.text:NmiSR)
                  00000dde    00000002     rtsv7M4_T_le_v4SPD16_eabi.lib : i_div0.obj (.text)
                  00000de0    00000002                                   : mpu_init.obj (.text)
                  00000de2    00000002                                   : startup.obj (.text)

.const     0    00000de4    000002fc     
                  00000de4    000001b0     driverlib.lib : sysctl.obj (.const:g_pppui32XTALtoVCO)
                  00000f94    00000090                   : gpio.obj (.const:g_pui32GPIOBaseAddrs)
                  00001024    0000006c                   : sysctl.obj (.const:g_pui32Xtals)
                  00001090    00000030                   : sysctl.obj (.const:g_sXTALtoMEMTIM)
                  000010c0    0000000c     uartstdio.obj (.const:g_ui32UARTBase)
                  000010cc    0000000c     uartstdio.obj (.const:g_ui32UARTPeriph)
                  000010d8    00000008     driverlib.lib : sysctl.obj (.const)

.cinit     0    000010e0    00000024     
                  000010e0    00000011     (.cinit..data.load) [load image, compression = lzss]
                  000010f1    00000003     --HOLE-- [fill = 0]
                  000010f4    00000008     (__TI_handler_table)
                  000010fc    00000008     (__TI_cinit_table)

.init_array 
*          0    00000000    00000000     UNINITIALIZED

.stack     0    20000000    00000200     UNINITIALIZED
                  20000000    00000200     --HOLE--

.data      0    20000200    00000020     UNINITIALIZED
                  20000200    0000000c     rtsv7M4_T_le_v4SPD16_eabi.lib : exit.obj (.data:$O1$$)
                  2000020c    00000008                                   : _lock.obj (.data:$O1$$)
                  20000214    00000005     uartstdio.obj (.data)
                  20000219    00000003     --HOLE--
                  2000021c    00000004     rtsv7M4_T_le_v4SPD16_eabi.lib : stkdepth_vars.obj (.data)

MODULE SUMMARY

       Module                     code   ro data   rw data
       ------                     ----   -------   -------
    .\
       startup_ccs.obj            12     512       0      
       spi_master.obj             324    0         0      
    +--+--------------------------+------+---------+---------+
       Total:                     336    512       0      
                                                          
    .\utils\
       uartstdio.obj              684    24        5      
    +--+--------------------------+------+---------+---------+
       Total:                     684    24        5      
                                                          
    C:/TI/TivaWare_C_Series-2.1.4.178/driverlib/ccs/Debug/driverlib.lib
       sysctl.obj                 668    596       0      
       gpio.obj                   456    144       0      
       ssi.obj                    146    0         0      
       uart.obj                   6      0         0      
    +--+--------------------------+------+---------+---------+
       Total:                     1276   740       0      
                                                          
    C:\TI\ccsv7\tools\compiler\ti-cgt-arm_16.9.1.LTS\lib\rtsv7M4_T_le_v4SPD16_eabi.lib
       memcpy_t2.obj              156    0         0      
       autoinit.obj               112    0         0      
       copy_decompress_lzss.obj   104    0         0      
       exit.obj                   84     0         12     
       boot.obj                   84     0         0      
       cpy_tbl.obj                76     0         0      
       u_divt2.obj                64     0         0      
       _lock.obj                  20     0         8      
       args_main.obj              24     0         0      
       copy_decompress_none.obj   14     0         0      
       pre_init.obj               4      0         0      
       stkdepth_vars.obj          0      0         4      
       i_div0.obj                 2      0         0      
       mpu_init.obj               2      0         0      
       startup.obj                2      0         0      
    +--+--------------------------+------+---------+---------+
       Total:                     748    0         24     
                                                          
       Stack:                     0      0         512    
       Linker Generated:          0      33        0      
    +--+--------------------------+------+---------+---------+
       Grand Total:               3044   1309      541    


LINKER GENERATED COPY TABLES

__TI_cinit_table @ 000010fc records: 1, size/record: 8, table size: 8
	.data: load addr=000010e0, load size=00000011 bytes, run addr=20000200, run size=00000020 bytes, compression=lzss


LINKER GENERATED HANDLER TABLE

__TI_handler_table @ 000010f4 records: 2, size/record: 4, table size: 8
	index: 0, handler: __TI_decompress_lzss
	index: 1, handler: __TI_decompress_none


GLOBAL SYMBOLS: SORTED ALPHABETICALLY BY Name 

address   name                           
-------   ----                           
00000a3d  C$$EXIT                        
00000cb1  GPIODirModeSet                 
000005eb  GPIOPadConfigSet               
00000b29  GPIOPinConfigure               
00000d45  GPIOPinTypeSSI                 
00000d57  GPIOPinTypeUART                
00000a91  InitConsole                    
00000dcd  ResetISR                       
UNDEFED   SHT$$INIT_ARRAY$$Base          
UNDEFED   SHT$$INIT_ARRAY$$Limit         
00000d69  SSIAdvDataPutFrameEnd          
00000da7  SSIAdvFrameHoldEnable          
00000d9b  SSIAdvModeSet                  
00000dc5  SSIBusy                        
00000c41  SSIConfigSetExpClk             
00000d7b  SSIDataGetNonBlocking          
00000db1  SSIDataPut                     
00000dbb  SSIEnable                      
00000201  SysCtlClockFreqSet             
00000c7d  SysCtlPeripheralEnable         
00000dd3  UARTClockSourceSet             
00000989  UARTStdioConfig                
00000cfd  UARTprintf                     
00000401  UARTvprintf                    
00000b71  UARTwrite                      
20000200  __STACK_END                    
00000200  __STACK_SIZE                   
20000200  __STACK_TOP                    
000010fc  __TI_CINIT_Base                
00001104  __TI_CINIT_Limit               
000010f4  __TI_Handler_Table_Base        
000010fc  __TI_Handler_Table_Limit       
000008b1  __TI_auto_init                 
20000200  __TI_cleanup_ptr               
00000921  __TI_decompress_lzss           
00000d8d  __TI_decompress_none           
20000204  __TI_dtors_ptr                 
20000208  __TI_enable_exit_profile_output
ffffffff  __TI_pprof_out_hndl            
ffffffff  __TI_prof_data_size            
ffffffff  __TI_prof_data_start           
00000000  __TI_static_base__             
00000ddf  __aeabi_idiv0                  
00000815  __aeabi_memcpy                 
00000815  __aeabi_memcpy4                
00000815  __aeabi_memcpy8                
00000c01  __aeabi_uidiv                  
00000c01  __aeabi_uidivmod               
ffffffff  __binit__                      
ffffffff  __c_args__                     
00000de1  __mpu_init                     
20000000  __stack                        
00000d19  _args_main                     
000009e9  _c_int00                       
2000020c  _lock                          
00000d3f  _nop                           
00000d37  _register_lock                 
00000d31  _register_unlock               
00000de3  _system_post_cinit             
00000dd9  _system_pre_init               
20000210  _unlock                        
00000a41  abort                          
ffffffff  binit                          
00000add  copy_in                        
00000a49  exit                           
00000000  g_pfnVectors                   
0000071d  main                           
2000021c  main_func_sp                   
00000815  memcpy                         


GLOBAL SYMBOLS: SORTED BY Symbol Address 

address   name                           
-------   ----                           
00000000  __TI_static_base__             
00000000  g_pfnVectors                   
00000200  __STACK_SIZE                   
00000201  SysCtlClockFreqSet             
00000401  UARTvprintf                    
000005eb  GPIOPadConfigSet               
0000071d  main                           
00000815  __aeabi_memcpy                 
00000815  __aeabi_memcpy4                
00000815  __aeabi_memcpy8                
00000815  memcpy                         
000008b1  __TI_auto_init                 
00000921  __TI_decompress_lzss           
00000989  UARTStdioConfig                
000009e9  _c_int00                       
00000a3d  C$$EXIT                        
00000a41  abort                          
00000a49  exit                           
00000a91  InitConsole                    
00000add  copy_in                        
00000b29  GPIOPinConfigure               
00000b71  UARTwrite                      
00000c01  __aeabi_uidiv                  
00000c01  __aeabi_uidivmod               
00000c41  SSIConfigSetExpClk             
00000c7d  SysCtlPeripheralEnable         
00000cb1  GPIODirModeSet                 
00000cfd  UARTprintf                     
00000d19  _args_main                     
00000d31  _register_unlock               
00000d37  _register_lock                 
00000d3f  _nop                           
00000d45  GPIOPinTypeSSI                 
00000d57  GPIOPinTypeUART                
00000d69  SSIAdvDataPutFrameEnd          
00000d7b  SSIDataGetNonBlocking          
00000d8d  __TI_decompress_none           
00000d9b  SSIAdvModeSet                  
00000da7  SSIAdvFrameHoldEnable          
00000db1  SSIDataPut                     
00000dbb  SSIEnable                      
00000dc5  SSIBusy                        
00000dcd  ResetISR                       
00000dd3  UARTClockSourceSet             
00000dd9  _system_pre_init               
00000ddf  __aeabi_idiv0                  
00000de1  __mpu_init                     
00000de3  _system_post_cinit             
000010f4  __TI_Handler_Table_Base        
000010fc  __TI_CINIT_Base                
000010fc  __TI_Handler_Table_Limit       
00001104  __TI_CINIT_Limit               
20000000  __stack                        
20000200  __STACK_END                    
20000200  __STACK_TOP                    
20000200  __TI_cleanup_ptr               
20000204  __TI_dtors_ptr                 
20000208  __TI_enable_exit_profile_output
2000020c  _lock                          
20000210  _unlock                        
2000021c  main_func_sp                   
ffffffff  __TI_pprof_out_hndl            
ffffffff  __TI_prof_data_size            
ffffffff  __TI_prof_data_start           
ffffffff  __binit__                      
ffffffff  __c_args__                     
ffffffff  binit                          
UNDEFED   SHT$$INIT_ARRAY$$Base          
UNDEFED   SHT$$INIT_ARRAY$$Limit         

[69 symbols]
